:100000000C949C000C94AE000C94AE000C94AE00CA
:100010000C94AE000C94AE000C94AE000C94AE00A8
:100020000C94AE000C94AE000C94AE000C94D60070
:100030000C9447040C94AE000C94AE000C94AE00EB
:100040000C94AE000C94AE000C94AE000C94AE0078
:100050000C94AE000C94AE000C94AE000C94AE0068
:100060000C94AE000C94AE000C94AE000C94AE0058
:100070000C94AE0000010000FE001200020000DC43
:1000800000220022000010012200210000EE0009E1
:1000900000030000D8000401030904CA000C020395
:1000A0000904BA000E03030904AC000C0C035B0046
:1000B0007300650072005D0000000E035B007000BD
:1000C00072006F0064005D0000000C035B006D00B7
:1000D000660067005D0000000403090409022900AE
:1000E000010100C000090400000103000000092113
:1000F00001010001222200070583034000011201D3
:10010000100100000040CDAB04F101010102030128
:1001100006C9FF0904A15C7508150026FF0095407B
:10012000097581029540097691029600020976B11F
:1001300002C0000001C1320011241FBECFEFD4E085
:10014000DEBFCDBF21E0A0E0B1E001C01D92A53A25
:10015000B207E1F70E94A7050C94EA050C94000091
:100160008091E80080FFFCCF08958091E80082FF35
:10017000FCCF0895E1E6F0E080E8808310820895E6
:100180008FEF8093A40180EA8093D80010926300DF
:1001900086E089BD09B400FEFDCF80E88093D800D9
:1001A0001092E0008CE08093E20008951F920F927D
:1001B0000FB60F9211242F938F939F939091E90084
:1001C0008091E1001092E10083FF11C01092E900DC
:1001D00081E08093EB001092EC0022E32093ED008D
:1001E00028E02093F000109203018093A4019093E3
:1001F000E9009F918F912F910F900FBE0F901F904C
:1002000018952F923F928F929F92AF92BF92CF926A
:10021000DF92EF92FF920F931F93CF93DF93CDB7AF
:10022000DEB7C054D1090FB6F894DEBF0FBECDBF04
:100230007C010E94B500539A5B9867018FE3C82246
:10024000DD249BB08FEF8AB966E0F694E7946A9557
:10025000E1F7FE01E05CFF4F5F017BEF872EE114C9
:10026000F10409F4E6C21091F100012F092910955B
:1002700019219091F1009A8350E8252E2220C1F097
:10028000822D89230BB9882359F0269400000000A1
:100290000000000000000000000000001BB9EECFCD
:1002A00000001BB926940000000000000000E6CF0B
:1002B0009091F1009B838091F1008C838091F100FB
:1002C0008D838091F1008E838091F1008F838091E6
:1002D000F10088878091F100898740E8242E222050
:1002E000C1F0822D89230BB9882359F02694000090
:1002F00000000000000000000000000000001BB92A
:10030000EECF00001BB926940000000000000000A2
:10031000E6CF8091F1008A878091F1008B878091F0
:10032000F1008C878091F1008D8730E8232E9C812D
:100330002220C1F0822D89230BB9882359F02694FD
:1003400000000000000000000000000000000000AD
:100350001BB9EECF00001BB926940000000000007E
:100360000000E6CF8091F1008E878091F1008F87A9
:100370008091F100888B8091F100898B8091F10050
:100380008A8B20E8222E9D812220C1F0822D892394
:100390000BB9882359F026940000000000000000EB
:1003A00000000000000000001BB9EECF00001BB9E8
:1003B00026940000000000000000E6CF8091F100CC
:1003C0008B8B8091F1008C8B8091F1008D8B8091D3
:1003D000F1008E8B90E8292E9E812220C1F0822D83
:1003E00089230BB9882359F02694000000000000EF
:1003F000000000000000000000001BB9EECF00006C
:100400001BB926940000000000000000E6CF809198
:10041000F1008F8B8091F100888F8091F100898F9E
:1004200080E8282E9F812220C1F0822D89230BB9DC
:10043000882359F02694000000000000000000000E
:100440000000000000001BB9EECF00001BB926948D
:100450000000000000000000E6CF8091F1008A8FCC
:100460008091F1008B8F8091F1008C8FB0E82B2E62
:1004700098852220C1F0822D89230BB9882359F059
:1004800026940000000000000000000000000000B2
:1004900000001BB9EECF00001BB92694000000003D
:1004A00000000000E6CF8091F1008D8F8091F10077
:1004B0008E8F8091F1008F8F8091F10088A3A0E84A
:1004C0002A2E99852220C1F0822D89230BB98823F9
:1004D00059F0269400000000000000000000000019
:1004E000000000001BB9EECF00001BB926940000ED
:1004F000000000000000E6CF8091F10089A3809108
:10050000F1008AA38091F1008BA38091F1008CA36C
:10051000F0E82F2E9A852220C1F0822D89230BB975
:10052000882359F02694000000000000000000001D
:100530000000000000001BB9EECF00001BB926949C
:100540000000000000000000E6CF8091F1008DA3C4
:100550008091F1008EA38091F1008FA38091F10032
:1005600088A7E0E82E2E9B852220C1F0822D8923CA
:100570000BB9882359F02694000000000000000009
:1005800000000000000000001BB9EECF00001BB906
:1005900026940000000000000000E6CF8091F100EA
:1005A00089A78091F1008AA78091F1008BA78091A3
:1005B000F1008CA770E8272E9C852220C1F0822DA7
:1005C00089230BB9882359F026940000000000000D
:1005D000000000000000000000001BB9EECF00008A
:1005E0001BB926940000000000000000E6CF8091B7
:1005F000F1008DA78091F1008EA78091F1008FA767
:100600008091F10088AB60E8262E9D852220C1F004
:10061000822D89230BB9882359F02694000000000D
:100620000000000000000000000000001BB9EECF39
:1006300000001BB926940000000000000000E6CF77
:100640008091F10089AB8091F1008AAB8091F1003B
:100650008BAB8091F1008CAB50E8252E9E8522203B
:10066000C1F0822D89230BB9882359F0269400000C
:1006700000000000000000000000000000001BB9A6
:10068000EECF00001BB9269400000000000000001F
:10069000E6CF8091F1008DAB8091F1008EAB80911F
:1006A000F1008FAB8091F10088AF40E8242E9F8548
:1006B0002220C1F0822D89230BB9882359F026947A
:1006C000000000000000000000000000000000002A
:1006D0001BB9EECF00001BB92694000000000000FB
:1006E0000000E6CF8091F10089AF8091F1008AAFE0
:1006F0008091F1008BAF8091F1008CAF30E8232E18
:1007000098892220C1F0822D89230BB9882359F0C2
:10071000269400000000000000000000000000001F
:1007200000001BB9EECF00001BB9269400000000AA
:1007300000000000E6CF8091F1008DAF8091F100C4
:100740008EAF8091F1008FAF8091F100F501808331
:1007500020E8222E99892220C1F0822D89230BB90D
:10076000882359F0269400000000000000000000DB
:100770000000000000001BB9EECF00001BB926945A
:100780000000000000000000E6CFF2E0EF16F104E8
:1007900010F08092E800FE01729690E8292E919167
:1007A0002220C1F0822D89230BB9882359F0269489
:1007B0000000000000000000000000000000000039
:1007C0001BB9EECF00001BB926940000000000000A
:1007D0000000E6CF85E18A95F1F70000EA15FB05F8
:1007E000E1F692E0E916F10410F00E94B50080E80D
:1007F000282EF50190812220C1F0822D89230BB98A
:10080000882359F02694000000000000000000003A
:100810000000000000001BB9EECF00001BB92694B9
:100820000000000000000000E6CFF1E0EF1AF10840
:1008300016CDC114D10429F08BEF8093E8000E94FB
:10084000B5005B9880E090E08C159D0521F020912B
:10085000F1000196F9CF8BEF8093E8008EEF809343
:10086000E800C05CDF4F0FB6F894DEBF0FBECDBF0F
:10087000DF91CF911F910F91FF90EF90DF90CF907C
:10088000BF90AF909F908F903F902F9008951F92B0
:100890000F920FB60F921124EF92FF920F931F93B6
:1008A0002F933F934F935F936F937F938F939F9378
:1008B000AF93BF93EF93FF93CF93DF931F92CDB787
:1008C000DEB71092E9008091E80083FF25C12091F6
:1008D000F1009091F100E090F1008091F100F12C95
:1008E000F82A8091F1003091F1000091F1004091DF
:1008F000F10010E0142B42EF4093E800963009F02D
:1009000047C090E0932B48E024E730E0F90165917F
:1009100074916E157F0539F4F901329665917491E1
:100920006817790729F0295F3F4F415079F7F4C0E4
:10093000F901349645915491F901369624910F3F6F
:10094000110519F010F00FEF10E0021708F4202F36
:100950003EEF8091E800982F9570D9F382FDDFC0BB
:10096000822F213408F080E4FA01982F992331F086
:1009700064916093F10091503196F8CF480F511D6A
:10098000281B3093E8002111E4CF803411F3C7C055
:10099000953051F48EEF8093E8000E94B0008E2DC8
:1009A00080688093E300BBC0993071F52111B0C01D
:1009B000E09203018EEF8093E80041E082E391E052
:1009C0004093E9009C012F5F3F4FFC0154915093ED
:1009D000EB00552359F0F90124912093EC009C0180
:1009E0002D5F3F4F319684918093ED004F5F4530EE
:1009F00011F0C901E5CF8EE18093EA001092EA0080
:100A000082E08093A4018BC0983041F4203809F033
:100A100083C00E94B0008091030137C0911107C0CC
:100A20000E94B0001092F1001092F1006DC097305A
:100A300021F40E94B0008AEA28C0933A81F48091A0
:100A4000E800982F9570D9F382FD69C08BE0809300
:100A5000F1008150E1F78EEF8093E8005DC0943A99
:100A6000B9F40E94B00034E03093F10025E0209307
:100A7000F10096E09093F10087E08093F1003093CD
:100A8000F1002093F1009093F1008093F1003CC0BD
:100A9000963A39F580E890E06EEF2091E800322F29
:100AA0003570D9F322FD3BC09C018134910510F0D3
:100AB00020E430E0422F442351F05091020171E0D4
:100AC000750F709302015093F1004150F4CF821BD7
:100AD000930B6093E800009701F720343105E9F2A9
:100AE0001EC0953AC9F40E94B50080E090E08017DE
:100AF000910739F02091F1002983298129830196FA
:100B0000F6CF8BEF8093E8008EEF8093E80007C06C
:100B1000C8010E94010103C081E28093EB000F90A5
:100B2000DF91CF91FF91EF91BF91AF919F918F9105
:100B30007F916F915F914F913F912F911F910F91F5
:100B4000FF90EF900F900FBE0F901F901895F894A4
:100B500081E08AB90E94BA000E94C0007894E4E261
:100B6000F1E080E381938F5F803BE1F72FEF89E62F
:100B700098E1215080409040E1F700C000002FEF45
:100B800089E698E1215080409040E1F700C00000E4
:100B90008091A4018230E4F333E04AEA5AE3F89406
:100BA0002091E9003093E9008091E80085FF08C0BA
:100BB00080E490E04093F1000197E1F75093E80062
:100BC0002093E90078948FE99FE00197F1F700C046
:080BD0000000E5CFF894FFCF0F
:00000001FF
